:020000040000FA
:1000000090040020D50000005B08000059080000A3
:1000100000000000000000000000000000000000E0
:10002000000000000000000000000000C10A000005
:100030000000000000000000950A0000C50A000052
:10004000E70000009D080000E7000000E700000056
:10005000E7000000E7000000E7000000E700000004
:10006000E7000000E7000000E7000000E7000000F4
:10007000E70000000000000000000000E7000000B2
:10008000E700000000000000E7000000E7000000BB
:1000900000000000E700000000000000710C0000FC
:1000A000E7000000E7000000000000000000000082
:1000B000E7000000E700000000000000E70000008B
:1000C0000348854600F000F900480047051100008C
:1000D000900400200448804704480047FEE7FEE7FC
:1000E000FEE7FEE7FEE7FEE7FD0A0000C1000000B4
:1000F00030B50B46014600202022012409E00D46C0
:10010000D5409D4205D31D469540491B2546954047
:1001100040191546521E002DF1DC30BD70B5024667
:100120004A40D50F40004A00ED0740085208002819
:1001300014D0002A12D0C40DD30D41020120C005F5
:100140005202490A520AE41A091812187D349142DF
:1001500001D3641C00E04900002C01DA002070BDCE
:100160000023914201D3891A034340084900002823
:10017000F7D100290AD0914202D10121C90705E037
:10018000914201D2012101E00121C943E005C018DB
:10019000401900F058F870BD420005D04200120E20
:1001A00052428A4201DB00207047C9050818704797
:1001B00010B500229623114600F04DF810BD410005
:1001C00040020122400AD205090E80187F2901DA77
:1001D00000207047962903DC9622511AC8407047C8
:1001E000963988407047C20FD207400040080BD0B4
:1001F000C10D0723DB01C91840020905400A11435C
:10020000C208400711437047002001467047CB0FDA
:10021000DB07490010B5490802460A4307D00A0D1A
:1002200007240903E401090B121B002A01DC00204A
:1002300010BDC900440F0C43C100E018D20580185E
:1002400000F001F810BD002904DA401C490001D17A
:1002500040084000704770B40024050C05D11024FC
:10026000000402D1002921D01124050E01D1000281
:100270000834050F01D10001241D850F01D1800034
:10028000A41C002801DB4000641C002908D02025A4
:100290002E1B0D46F540A14000D001212943084303
:1002A00001061B1B000ADB1D02D5002070BC704735
:1002B000DB05181880180029F8DA401C4900F5D130
:1002C00070BC400840007047064C0125064E05E012
:1002D000E36807CC2B430C3C98471034B442F7D367
:1002E000FFF7F2FE181800003818000001218907F6
:1002F0000868C007C00F01D0054A0A600022054BFC
:10030000D2439A60002801D00020086070470000A6
:100310009669AA554000004000B5030000F06EFD4C
:100320002B171945454545454527292B2D2F314587
:10033000191B1D1F21232527292B2D2F313335373D
:100340004545454545393B3D3F4541434500002036
:1003500000BD012000BD022000BD032000BD04201F
:1003600000BD052000BD062000BD072000BD0820FF
:1003700000BD092000BD0A2000BD0B2000BD0C20DF
:1003800000BD0D2000BD0E2000BD0F2000BD1020BF
:1003900000BD162000BD172000BD182000BD19208B
:1003A00000BD1B2000BD1C2000BDFF2000BD30B5DE
:1003B000054608780C4601280FD00021284600F099
:1003C000DBF9A178284600F073F86178284600F040
:1003D00059F86078002812D019E00121284600F071
:1003E000CBF90121284600F04DF80021284600F005
:1003F0005FF80021284600F077F9002110E021790C
:10040000284600F027F8E178284600F03DF9012160
:10041000284600F099F96179284600F065F9A1793C
:10042000284600F049F90021284600F075F930BD52
:1004300000B50146FFF770FF0D2901D8044901E01E
:10044000034980390968C140C807C00F00BD0000DA
:100450008004004010B50446FFF75EFF01220D2C1A
:1004600003D8074B03E0596010BD054B803B0029C2
:10047000596802D082401143F5E782409143F2E788
:10048000C004004010B50446FFF746FF01220D2CC2
:1004900007D8064B07E082409A6110BD8240DA61BE
:1004A00010BD024B803B0129F8D1F4E780040040E5
:1004B000F0B5002906D0012904D0022902D0032971
:1004C00000D0FF2130256F4A6E4C2E022F03803A58
:1004D000030000F093FC2B171D2323232323232445
:1004E0002A2F363B4023494E555A5F666D767C81F4
:1004F000888D9299A0A92323232323AFB6BFC523B8
:10050000CACF2300606A890780088000890F03E052
:10051000606A8907A843890E08436062F0BDA06A3B
:10052000890780088000890F1BE0A06A8907A8431B
:10053000890E16E0A06A0322120290438907890DF2
:100540000FE0A06A8907B043890C0AE0A06A890716
:10055000B843890B05E0A06A03221205904389077E
:10056000890A0843A062F0BD506A8907A843890E32
:1005700024E0506A03231B0298438907890D1DE07C
:10058000506A8907B043890C18E0506A8907B8435C
:10059000890B13E0506A03231B0598438907890AD6
:1005A0000CE0506A03231B0698438907890905E07C
:1005B000506A03231B079843890789080843506240
:1005C000F0BD906A890780088000890F29E0906A51
:1005D0008907A843890E24E0906A03231B029843ED
:1005E0008907890D1DE0906A8907B043890C18E0DE
:1005F000906A8907B843890B13E0906A03231B05AF
:1006000098438907890A0CE0906A03231B069843E4
:100610008907890905E0906A03231B079843890726
:10062000890808439062F0BDD06A8907800880007D
:10063000890F0CE0D06A03231B06984389078909B8
:1006400005E0D06A03231B079843890789080843FC
:10065000D062F0BD106B890780088000890F0DE023
:10066000106B8907A843890E08E0106B8907B04317
:10067000890C03E0106B8907B843890B08431063AA
:10068000F0BD00008004004010B50446FFF744FEB2
:1006900001220D2C03D8074B03E0996310BD054BD5
:1006A000803B0029996B02D082401143F5E78240DC
:1006B0009143F2E78004004010B50446FFF72CFE9A
:1006C00001220D2C03D8074B03E0196010BD054B28
:1006D000803B0029196802D082401143F5E782402F
:1006E0009143F2E7C004004010B50446FFF714FE42
:1006F00001220D2C03D8074B03E0D96310BD054B35
:10070000803B0029D96B02D082401143F5E782403B
:100710009143F2E78004004010B50446FFF7FCFD6A
:1007200001220D2C03D8074B03E0D96010BD054B07
:10073000803B0029D96802D082401143F5E782400E
:100740009143F2E7C004004010B50446FFF7E4FD12
:1007500001220D2C03D8074B03E0996010BD054B17
:10076000803B0029996802D082401143F5E782401E
:100770009143F2E7C004004010B50446FFF7CCFDFA
:1007800001220D2C03D8074B03E0596310BD054B24
:10079000803B0029596B02D082401143F5E782402B
:1007A0009143F2E78004004010B50446FFF7B4FD22
:1007B00001220D2C07D8064B07E082409A6010BD3D
:1007C0008240DA6010BD024B803B0129F8D1F4E78A
:1007D0008004004030B501241D4BA407236002258E
:1007E0001C4B012858680DD04008400058605868DC
:1007F000A8435860186880088000401C18600020DA
:10080000206030BD800309D458684008400058601B
:1008100058682843586058688003FCD5206A00094E
:100820000001401C206258680C258907A843090F65
:1008300008435860012A03D058688003FCD5DEE7DE
:10084000186880088000186058688003FCD5D6E7D7
:100850009669AA5540000040FEE7704730B5C406CF
:10086000E40E0123A340002A10D08408094AA40002
:10087000A21814688007C00EFF2585408907090E5D
:10088000AC43814021431160034801E002488030BD
:10089000036030BD00E400E000E100E010B50F208F
:1008A00000F00CF8012807D10F2000F013F8012800
:1008B00002D10F2000F048F810BD000000B500F094
:1008C00015F803494968C140C807C00F00BD0000C2
:1008D0000007004000B500F009F803490968C1406D
:1008E000C807C00F00BD00000007004000B50300AE
:1008F00000F084FA2B171927272727272717191BFA
:100900001D1F2127191B1D1F21232517191B1D1F03
:1009100021232517272727272723251719271D1FB9
:100920002700002000BD012000BD022000BD0320E3
:1009300000BD042000BD052000BD062000BD07202D
:1009400000BDFF2000BD000000B5FFF7CFFF034949
:1009500009680904C140C801C00F00BD000700407C
:1009600000B5030000F04AFA2B1F1F232323232383
:1009700023212121212121231717171717171719B1
:10098000191919191919191B23232323231B1B1D9B
:100990001D231D1D2300002000BD012000BD0220DD
:1009A00000BD032000BD042000BD052000BDFF20C8
:1009B00000BD30B50C460546497800F033F8217883
:1009C000284600F001F830BD70B50446FFF78EFFF1
:1009D00002462046FFF7C4FF104B04469D68900076
:1009E00007268640B54384402C439C600125284659
:1009F000904058601C68002908D001460832214305
:100A00009540A94319600649086070BD08328443C7
:100A1000954025431D6002498031F5E700070040FD
:100A200000E100E010B5FFF761FF0C4CE2688000C8
:100A3000072383409A430B0000F0E0F90509040600
:100A40000B0D0900012100E0022181400A43E26010
:100A500010BD0321F9E70421F7E70000000700407B
:100A60003EB50024684604700125457084704471C9
:100A7000857169460F20FFF79AFC6846057244723B
:100A800002A90F20FFF795FF012211461046FFF73C
:100A9000E5FE3EBD704700000121074A89070A6054
:100AA000064A136880079B089B00800F034313606E
:100AB00000200860704700009669AA554000004079
:100AC0007047000002480168491C0160704700003F
:100AD00084000020084A0368002153619161037972
:100AE000002B00D0042143790220002B01D00143C8
:100AF00000E081431161704700E000E010B5002084
:100B0000FFF7CAFF10BD026906239A430B789B07C3
:100B10005B0F1A430261026908239A434B78DB0793
:100B20001B0F1A430261026930239A438B789B079B
:100B30009B0E1A4302610269C0239A43CB789B073C
:100B40001B0E1A430261C2680979120A1202491E79
:100B5000C9B20A43C26081698022914381617047B2
:100B60000169490849000161704701690122114387
:100B700001617047026903231B0389079A43890CAB
:100B80000A4302617047826903231B0389079A4362
:100B9000890C0A4382617047026903239B0389071A
:100BA0009A43090C0A4302617047826903239B033D
:100BB00089079A43090C0A438261704782690B785E
:100BC00052085200DB07DB0F1A438261826902235D
:100BD0009A434B78DB079B0F1A4382618269042397
:100BE0009A438B78DB075B0F1A4382618269082383
:100BF0009A43CB78DB071B0F1A438261826930234B
:100C00009A430B799B079B0E1A43826182694023AA
:100C10009A434B79DB075B0E1A43826182698979BB
:100C20008023C9079A43090E0A438261704703690A
:100C3000012212049343036143681B0C1B040B4302
:100C400043600169114301617047826B120C120409
:100C50000A4382637047C26B120C12040A43C263D8
:100C60007047426C120C12040A4342647047000041
:100C700010B5044C204600F089F80146204600F0EB
:100C800088F810BD00600040C16170470246D2691B
:100C900000200A4200D001207047012A826902D058
:100CA0008A43826170470A43FBE70000F8B50D46AE
:100CB0000E7B3449044600200F68012E06D0022E18
:100CC00007D0032E08D0042E09D013E0A868000135
:100CD00007E0A868400104E0A868800101E0A86876
:100CE000C001FFF765FA00903846FFF761FA0099F6
:100CF000FFF714FA7F21C905884202DA0020224951
:100D000001E0FFF770FAFFF782FA0421FFF744FAD7
:100D1000FFF755FA61680722120291437207520DDC
:100D200011436160206120680121490388432978CB
:100D3000C907890C0843206020680F2109028843F5
:100D400069780907090D084320602068012109031B
:100D50008843A978C907C90C0843206020680F217F
:100D600009068843E97809070909084320602068D3
:100D70000121090788432979C907C9080843206068
:100D8000F8BD0000800000200000F03F2030007916
:100D900070472030017070474268890792089200BE
:100DA000890F0A43426070471CB50A487D21C9007B
:100DB0000068FFF79DF900900120694608714871AD
:100DC0006846FFF787FE0448016949084900016148
:100DD0001CBD00008000002000E000E00FB410B552
:100DE00003A9044B044A029800F024F810BC08BC84
:100DF00004B01847850F00008800002030B4744606
:100E0000641E2578641CAB4200D21D46635D5B0006
:100E1000E31830BC184702E008C8121F08C1002AB6
:100E2000FAD170477047002001E001C1121F002A6B
:100E3000FBD17047FFB58DB00446002506E025289C
:100E40000AD0109A0F999047641C6D1C20780028D6
:100E5000F5D1284611B0F0BD00270121484A00977E
:100E600000E00743641C23780846203B984010426A
:100E7000F7D120782E2817D1042007436078641C0E
:100E80002A280CD10E98641C02C800910E900BE029
:100E900000990A22514330394018641C0090207890
:100EA000014630390929F3D920780028D1D06428A7
:100EB00008D0692806D075281ED0109A0F9990473F
:100EC0006D1C5BE00A200E99019001C90E9100286B
:100ED00002DA40422D2102E0390504D52B216A4671
:100EE0001172012103E0F90704D02021F7E70BAECE
:100EF0000B910DE00021FAE70A200E99019001C93B
:100F00000E91F7E70199FFF7F3F83031761E317053
:100F10000028F7D103A8801B20300190780701D565
:100F2000009801E0012000900199884201DD401AFB
:100F300000E000200027009006E002A8109AC05DA3
:100F40000F9990476D1C7F1C0B988742F5DB04E0DE
:100F5000109A30200F9990476D1C0099481E009000
:100F60000029F5DC05E03078109A761C0F9990473F
:100F70006D1C0199481E01900029F4DC641C65E792
:100F800009280100F8B50E4F0646C1B200243846C4
:100F9000FFF7FFFE0B4D02213846FFF777FE641C7A
:100FA000002801D1AC42F6D102213846FFF76CFE91
:100FB000AC4202D10020C043F8BD3046F8BD00006D
:100FC00000600040E21C000070B5094C0021606820
:100FD00000F0A8FA00250320A56000F00BF804201B
:100FE00000F01AFB65610020E56000F089F970BD32
:100FF0000000002010B500280AD001280AD00228DD
:1010000010D0032817D1002000F0D8F9002005E007
:101010000120F9E7002000F0D1F9012000F0C7F924
:10102000002006E0002000F0C9F9002000F0BFF920
:10103000012000F0B5F910BD10B500F037F800F050
:101040001FF8FFF70DFD10BD10B5084B186900F033
:101050006DF99969884207D3054800681861FFF760
:10106000B3FF04A0FFF7BAFE10BD0000000000208F
:101070008400002074696D65206F7665720D0A002A
:101080001CB500206A46107001215170907050719B
:10109000917169461920FFF78AF969461E20FFF70A
:1010A00086F969461B20FFF782F91CBD1CB500209C
:1010B000694600900871487188711120FFF777F92F
:1010C00069460D20FFF773F969461320FFF76FF9A2
:1010D00069461420FFF76BF969461520FFF767F999
:1010E00069461620FFF763F969461720FFF75FF995
:1010F00069460120FFF75BF969462A20FFF757F997
:101100001CBD0000012203211046FFF763FBFFF71F
:10111000F5FCFFF7EBF8FFF747FE114908690122DC
:101120001043086100F0A8FAFFF786FF0D4800F0B1
:10113000FDFA00F025FA0020FFF75CFF012000F027
:10114000DFF809A0FFF74AFE064C6C3C00F0BAF845
:1011500000F0F8F8A0680228F8D1FFF775FFF5E76E
:1011600000E000E06C000020496E697469616C6900
:101170007A6174696F6E20636F6D706C65746564FD
:101180000D0A0000254A10B5012190420BD1437A87
:10119000002B08D1037C002B05D1C368962B02D30A
:1011A00001741FA037E090420FD1427A022A0CD17D
:1011B000027C002A09D1C268962A06D801741CA0B4
:1011C000FFF70CFE00F048F910BD144A1C329042A3
:1011D00012D1427A012A0FD1027C002A0CD1C268B6
:1011E000962A09D8017418A0FFF7F8FD0B48343887
:1011F000C06800F0EBF810BD084A38329042FAD1CE
:10120000427A012AF7D1027C002AF4D1C268962AD8
:10121000F1D8017412A0FFF7E1FD10BD34000020E9
:101220006B657930207A6B735F6B6565700D0A00B2
:101230006B657930207A6B735F66616C6C696E6781
:101240005F656467650D0A006B657931207A6B73A1
:101250005F726973696E675F656467650D0A000098
:101260006B657932207A6B735F726973696E675F41
:10127000656467650D0A000010B501210C4A04463B
:101280000846916000F03CF8002C08D0012C08D0F2
:10129000022C08D0032C01D1FFF796FE10BD0020D0
:1012A00002E0012000E00220FFF7A4FE10BD0000D4
:1012B00000000020012110B541402A20FFF774FAF8
:1012C00010BD000010B50C4BD86900F02FF87D213F
:1012D000C90088420CD909480068D86118780028EC
:1012E00007D000201870002800D00120FFF7E2FF8F
:1012F00010BD0120F6E7000000000020840000205F
:1013000010B501460120FFF74FFA10BD10B51E20A1
:10131000FFF78EF8012800D0002010BD10B519206D
:10132000FFF786F8012800D0002010BD01460448D0
:1013300002680068401A8A4200D2401E70470000CE
:101340008400002010B5064B186AFFF7EFFF142841
:1013500005D9044800681862002000F0D1F910BDDA
:101360000000002084000020012110B54140112020
:10137000FFF71AFA10BD012110B541400D20FFF70B
:1013800013FA10BD012110B541401320FFF70CFAEC
:1013900010BD012110B541401420FFF705FA10BD22
:1013A000012110B541401720FFF7FEF910BD0121C2
:1013B00010B541401620FFF7F7F910BD012110B517
:1013C00041401520FFF7F0F910BD000070B51D4C2D
:1013D00001001B4D606812D001291BD0022924D0C6
:1013E00003290BD1296800F09DF80020E06016A0C9
:1013F0002968FFF7F3FC0320FFF73EFF70BDE968A3
:1014000000F090F80120E0600FA0E968FFF7E6FC2B
:101410000020F1E7A96800F085F80220E0600AA04A
:10142000A968FFF7DBFC0120E6E7696800F07AF8BD
:101430000320E06004A06968FFF7D0FC0220DBE72E
:10144000240000200000002070776D20675F647525
:1014500074793A256400000070B5224CA068002819
:1014600001D1FFF7B3FF204802250068A560206185
:101470000120FFF745FF606901260300FFF7BEFC6E
:1014800005040C141D282700184919A0A161FFF7B5
:10149000A5FC0020666118E01B4915A0A161FFF7BB
:1014A0009DFC0120656110E0184911A0A161FFF7C2
:1014B00095FC03206061022007E015490CA0A161A2
:1014C000FFF78CFC04206061032000F0A5F870BDDC
:1014D00010A0A660FFF782FC042000F09DF8002019
:1014E000606170BD000000208400002080EE3600A6
:1014F000675F6F7A6F6E655F776F726B5F74696D30
:10150000653A2564000000000044950800E6DF0C01
:1015100000882A11636C6F73652074696D696E674A
:101520000000000070B50B4C05460E462046FFF744
:1015300017FB00F025F8B1B22046FFF786FB0648FE
:10154000808881B22046FFF786FBA9B22046FFF7CC
:1015500088FB70BD00200040000000201CB500206A
:101560006A461070507002219170D0701071012184
:101570005171907169461220FEF719FF1CBD0000E1
:101580007FB5002468460472447284720321C172DC
:101590001F4E012502A930460395FFF7B4FA6846AD
:1015A000047045708470C47004714471857169461B
:1015B0003046FFF703FB00213046FFF7DBFA02213C
:1015C0003046FFF7E9FA02213046FFF7DCFA012145
:1015D0003046FFF7EAFA00213046FFF728FB0D48B6
:1015E000808981B23046FFF730FB0A4C243CA0884A
:1015F00081B23046FFF72FFBA08881B23046FFF75B
:1016000030FBFFF7ABFF3046FFF7AFFA7FBD0000BE
:10161000002000402400002010B50300FFF7EEFB7F
:101620000504061119262500012020E00020FFF7FF
:101630009BFE0120FFF79FFE0020FFF7A3FE002086
:1016400011E00020FFF790FE0020FFF794FE01203C
:10165000F3E70020FFF788FE0020FFF78CFE002054
:10166000FFF790FE0120FFF794FE10BD0020FFF76A
:101670007BFE0020DEE7000070B586B000246846DF
:101680004470012505718570C470847144710470C3
:1016900069462520FEF78BFE68464570057185700A
:1016A000C47084714471047069462420FEF77FFE83
:1016B000E1204002049068460575C4720473047208
:1016C000447284720D4C02A92046FFF7EFFA012202
:1016D000160431462046FFF7E0FA00212046FFF7C6
:1016E0005BFB012211461720FFF7B8F8206828435A
:1016F000206020683043206006B070BD006000406C
:1017000070B5094D287800280CD0002406E0016847
:101710001C206043081800F02FF8641C68684168BA
:10172000A142F4DC70BD000078000020F8B5114F34
:10173000786001203870002417E01C2325465D43A3
:101740002B46026800210933D15400682E1D8059B0
:1017500080477968321D0B68985408688059804723
:10176000796811350968641C485578684168A14258
:10177000E3DCF8BD7800002010B50446C068401CCA
:10178000E060606880477D226169D200914201D2A9
:10179000491C6161217E814202D00021616103E028
:1017A0006169002900D060742076617C204600F0D9
:1017B00001F810BD70B50D460446017A0F480026A9
:1017C0004068A94211D0002D07D0E660267401219F
:1017D000617282682046904705E00221617282684A
:1017E00020469047E660257270BD31466672002D36
:1017F000FAD082682046904770BD00007800002033
:1018000074696D65726B65790000000067656172CF
:10181000736B65790000000038180000000000209C
:101820008C000000160E0000C41800008C00002080
:1018300004040000260E00000100000080BB000030
:101840000000000001000000000000000000000097
:101850000000000000000000000000000000000088
:10186000E02E0000C05D00007FBB000000180000FB
:101870001D13000000000000000000000000000038
:1018800000000000000000000C1800000D13000014
:101890000000000000000000000000000000000048
:1018A000000000003400002002000000851100004C
:1018B0000000000000000000006CDC0200000000DE
:0418C0000000000024
:04000005000000C136
:00000001FF
